
 WFWNET

 Start     Length     Name                   Class
 0001:0000 0215FH     _TEXT                  CODE
 0001:215F 000C1H     INIT_TEXT              CODE
 0001:2220 00000H     ints_TEXT              CODE
 0002:0000 003B1H     _DATA                  DATA
 0002:03B2 00000H     CONST                  CONST
 0002:03B2 00000H     _BSS                   BSS
 0002:03C0 0000CH     c_common               BSS

 Origin   Group
 0002:0   DGROUP

 Address   Export                  Alias

 0001:1EC4 DISABLE                 DISABLE
 0001:1EB2 ENABLE                  ENABLE
 0001:1BA0 I_AUTOLOGON             I_AUTOLOGON
 0001:1C10 I_CHANGECACHEPASSWORD   I_CHANGECACHEPASSWORD
 0001:1BEC I_CHANGEPASSWORD        I_CHANGEPASSWORD
 0001:1C34 I_CONNECTDIALOG         I_CONNECTDIALOG
 0001:1C58 I_CONNECTIONDIALOG      I_CONNECTIONDIALOG
 0001:1BC6 I_LOGOFF                I_LOGOFF
 0001:1F9E LFNCOPY                 LFNCOPY
 0001:1FE6 LFNDELETE               LFNDELETE
 0001:1F32 LFNFINDCLOSE            LFNFINDCLOSE
 0001:1EEA LFNFINDFIRST            LFNFINDFIRST
 0001:1F0E LFNFINDNEXT             LFNFINDNEXT
 0001:1F56 LFNGETATTRIBUTES        LFNGETATTRIBUTES
 0001:2052 LFNGETVOLUMELABEL       LFNGETVOLUMELABEL
 0001:200A LFNMKDIR                LFNMKDIR
 0001:1FC2 LFNMOVE                 LFNMOVE
 0001:209A LFNPARSE                LFNPARSE
 0001:202E LFNRMDIR                LFNRMDIR
 0001:1F7A LFNSETATTRIBUTES        LFNSETATTRIBUTES
 0001:2076 LFNSETVOLUMELABEL       LFNSETVOLUMELABEL
 0001:20BE LFNVOLUMETYPE           LFNVOLUMETYPE
 0001:1ED6 WEP                     WEP
 0001:012C WNETABORTJOB            WNETABORTJOB
 0001:0828 WNETADDCONNECTION       WNETADDCONNECTION
 0001:0E48 WNETBROWSEDIALOG        WNETBROWSEDIALOG
 0001:1C7C WNETCACHEPASSWORD       WNETCACHEPASSWORD
 0001:09BE WNETCANCELCONNECTION    WNETCANCELCONNECTION
 0001:0240 WNETCANCELJOB           WNETCANCELJOB
 0001:0068 WNETCLOSEJOB            WNETCLOSEJOB
 0001:0F40 WNETCONNECTDIALOG       WNETCONNECTDIALOG
 0001:107E WNETCONNECTIONDIALOG    WNETCONNECTIONDIALOG
 0001:04CE WNETDEVICEMODE          WNETDEVICEMODE
 0001:1722 WNETDIRECTORYNOTIFY     WNETDIRECTORYNOTIFY
 0001:0FE8 WNETDISCONNECTDIALOG    WNETDISCONNECTDIALOG
 0001:1CE8 WNETENUMCACHEDPASSWORDS  WNETENUMCACHEDPASSWORDS
 0001:1B7C WNETEXITCONFIRM         WNETEXITCONFIRM
 0001:1CA0 WNETGETCACHEDPASSWORD   WNETGETCACHEDPASSWORD
 0001:0690 WNETGETCAPS             WNETGETCAPS
 0001:0A92 WNETGETCONNECTION       WNETGETCONNECTION
 0001:160E WNETGETDIRECTORYTYPE    WNETGETDIRECTORYTYPE
 0001:1DE4 WNETGETERROR            WNETGETERROR
 0001:1E30 WNETGETERRORTEXT        WNETGETERRORTEXT
 0001:1DC0 WNETGETLASTCONNECTION   WNETGETLASTCONNECTION
 0001:1254 WNETGETPROPERTYTEXT     WNETGETPROPERTYTEXT
 0001:1D54 WNETGETSHARECOUNT       WNETGETSHARECOUNT
 0001:1D78 WNETGETSHARENAME        WNETGETSHARENAME
 0001:1D9C WNETGETSHAREPATH        WNETGETSHAREPATH
 0001:0D20 WNETGETUSER             WNETGETUSER
 0001:0188 WNETHOLDJOB             WNETHOLDJOB
 0001:03B6 WNETLOCKQUEUEDATA       WNETLOCKQUEUEDATA
 0001:0000 WNETOPENJOB             WNETOPENJOB
 0001:1AA2 WNETPRINTMGRCHANGEMENUS  WNETPRINTMGRCHANGEMENUS
 0001:1AC6 WNETPRINTMGRCOMMAND     WNETPRINTMGRCOMMAND
 0001:1AEA WNETPRINTMGREXITING     WNETPRINTMGREXITING
 0001:1B0C WNETPRINTMGREXTHELP     WNETPRINTMGREXTHELP
 0001:1B32 WNETPRINTMGRMOVEJOB     WNETPRINTMGRMOVEJOB
 0001:1A7E WNETPRINTMGRPRINTERENUM  WNETPRINTMGRPRINTERENUM
 0001:1A5A WNETPRINTMGRSELNOTIFY   WNETPRINTMGRSELNOTIFY
 0001:1B58 WNETPRINTMGRSTATUSCHANGE  WNETPRINTMGRSTATUSCHANGE
 0001:1172 WNETPROPERTYDIALOG      WNETPROPERTYDIALOG
 0001:0472 WNETQPOLL               WNETQPOLL
 0001:01E4 WNETRELEASEJOB          WNETRELEASEJOB
 0001:1CC4 WNETREMOVECACHEDPASSWORD  WNETREMOVECACHEDPASSWORD
 0001:0C2C WNETRESTORECONNECTION   WNETRESTORECONNECTION
 0001:153E WNETSERVERBROWSEDIALOG  WNETSERVERBROWSEDIALOG
 0001:1D30 WNETSETDEFAULTDRIVE     WNETSETDEFAULTDRIVE
 0001:029C WNETSETJOBCOPIES        WNETSETJOBCOPIES
 0001:1386 WNETSHAREASDIALOG       WNETSHAREASDIALOG
 0001:1D0C WNETSHARESDIALOG        WNETSHARESDIALOG
 0001:1462 WNETSTOPSHAREDIALOG     WNETSTOPSHAREDIALOG
 0001:041A WNETUNLOCKQUEUEDATA     WNETUNLOCKQUEUEDATA
 0001:035E WNETUNWATCHQUEUE        WNETUNWATCHQUEUE
 0001:02FA WNETWATCHQUEUE          WNETWATCHQUEUE

  Address         Publics by Name

 0000:0000  Imp  CALLPROC32W          (KERNEL.517)
 0001:1EC4       DISABLE
 0001:1EB2       ENABLE
 0001:173C       GETLASTERROR32
 0000:0000  Imp  GETMODULEUSAGE       (KERNEL.48)
 0000:0000  Imp  GETPROCADDRESS       (KERNEL.50)
 0000:0000  Imp  GETPROCADDRESS32W    (KERNEL.515)
 0000:0000  Imp  GETPROFILESTRING     (KERNEL.58)
 0000:0000  Imp  GETWINFLAGS          (KERNEL.132)
 0000:0000  Imp  GLOBALALLOC          (KERNEL.15)
 0000:0000  Imp  GLOBALFREE           (KERNEL.17)
 0000:0000  Imp  GLOBALLOCK           (KERNEL.18)
 0000:0000  Imp  GLOBALUNLOCK         (KERNEL.19)
 0001:21D3       GRABINTERRUPTS
 0000:0000  Imp  INITTASK             (KERNEL.91)
 0001:1BA0       I_AUTOLOGON
 0001:1C10       I_CHANGECACHEPASSWORD
 0001:1BEC       I_CHANGEPASSWORD
 0001:1C34       I_CONNECTDIALOG
 0001:1C58       I_CONNECTIONDIALOG
 0001:1BC6       I_LOGOFF
 0001:1F9E       LFNCOPY
 0001:1FE6       LFNDELETE
 0001:1F32       LFNFINDCLOSE
 0001:1EEA       LFNFINDFIRST
 0001:1F0E       LFNFINDNEXT
 0001:1F56       LFNGETATTRIBUTES
 0001:2052       LFNGETVOLUMELABEL
 0001:200A       LFNMKDIR
 0001:1FC2       LFNMOVE
 0001:209A       LFNPARSE
 0001:202E       LFNRMDIR
 0001:1F7A       LFNSETATTRIBUTES
 0001:2076       LFNSETVOLUMELABEL
 0001:20BE       LFNVOLUMETYPE
 0001:21A1       LibEntry
 0001:0750       LIBMAIN
 0000:0000  Imp  LOADLIBRARY          (KERNEL.95)
 0000:0000  Imp  LOADLIBRARYEX32W     (KERNEL.513)
 0000:0000  Imp  LocalInit            (KERNEL.4)
 0000:0000  Imp  LSTRCMP              (USER.430)
 0000:0000  Imp  LSTRCPY              (KERNEL.88)
 0000:0000  Imp  LSTRLEN              (KERNEL.90)
 0000:0000  Imp  OPENFILE             (KERNEL.74)
 0001:20E2       PmIpx2fHandler
 0001:2111       PmIpx73Handler
 0001:214D       PmIpxEntryPoint
 0001:10A0       PRINTCONNECTDIALOG
 0001:1ED6       WEP
 0001:012C       WNETABORTJOB
 0001:0828       WNETADDCONNECTION
 0001:0E48       WNETBROWSEDIALOG
 0001:1C7C       WNETCACHEPASSWORD
 0001:09BE       WNETCANCELCONNECTION
 0001:0240       WNETCANCELJOB
 0001:0068       WNETCLOSEJOB
 0001:0F40       WNETCONNECTDIALOG
 0001:107E       WNETCONNECTIONDIALOG
 0001:04CE       WNETDEVICEMODE
 0001:1722       WNETDIRECTORYNOTIFY
 0001:0FE8       WNETDISCONNECTDIALOG
 0001:1CE8       WNETENUMCACHEDPASSWORDS
 0001:1E78       WNETERRORTEXT
 0001:1B7C       WNETEXITCONFIRM
 0001:1CA0       WNETGETCACHEDPASSWORD
 0001:0690       WNETGETCAPS
 0001:0580       WNETGETCAPS16
 0001:0A92       WNETGETCONNECTION
 0001:160E       WNETGETDIRECTORYTYPE
 0001:1DE4       WNETGETERROR
 0001:05D6       WNETGETERROR16
 0001:1E30       WNETGETERRORTEXT
 0001:062E       WNETGETERRORTEXT16
 0001:1DC0       WNETGETLASTCONNECTION
 0001:1254       WNETGETPROPERTYTEXT
 0001:1D54       WNETGETSHARECOUNT
 0001:1D78       WNETGETSHARENAME
 0001:1D9C       WNETGETSHAREPATH
 0001:0D20       WNETGETUSER
 0001:0188       WNETHOLDJOB
 0001:03B6       WNETLOCKQUEUEDATA
 0001:0000       WNETOPENJOB
 0001:1AA2       WNETPRINTMGRCHANGEMENUS
 0001:1AC6       WNETPRINTMGRCOMMAND
 0001:1AEA       WNETPRINTMGREXITING
 0001:1B0C       WNETPRINTMGREXTHELP
 0001:1B32       WNETPRINTMGRMOVEJOB
 0001:1A7E       WNETPRINTMGRPRINTERENUM
 0001:1A5A       WNETPRINTMGRSELNOTIFY
 0001:1B58       WNETPRINTMGRSTATUSCHANGE
 0001:1172       WNETPROPERTYDIALOG
 0001:0472       WNETQPOLL
 0001:01E4       WNETRELEASEJOB
 0001:1CC4       WNETREMOVECACHEDPASSWORD
 0001:0C2C       WNETRESTORECONNECTION
 0001:153E       WNETSERVERBROWSEDIALOG
 0001:1D30       WNETSETDEFAULTDRIVE
 0001:029C       WNETSETJOBCOPIES
 0001:1386       WNETSHAREASDIALOG
 0001:1D0C       WNETSHARESDIALOG
 0001:1462       WNETSTOPSHAREDIALOG
 0001:041A       WNETUNLOCKQUEUEDATA
 0001:035E       WNETUNWATCHQUEUE
 0001:0524       WNETVIEWQUEUEDIALOG
 0001:02FA       WNETWATCHQUEUE
 0001:00CA       WNETWRITEJOB
 0000:0000  Imp  WRITEPROFILESTRING   (KERNEL.59)
 0001:1A3E       _FreeAlignedMemory
 0001:17B0       _Get32BitEntryPoints
 0001:19DA       _GetAlignedMemory
 0001:0704       _GetLanmanDrvEntryPoints
 0001:0802       _I_SetCapBits
 0000:0000  Imp  _LCLOSE              (KERNEL.81)
 0002:01EC       _lpfnClosePrinter
 0002:01F0       _lpfnConnectToPrinter
 0002:01E8       _lpfnGetLastError32
 0002:0014       _lpfnWNetAbortJob
 0002:01A8       _lpfnWNetAddConnection
 0002:01BC       _lpfnWNetBrowseDialog
 0002:01AC       _lpfnWNetCancelConnection
 0002:0020       _lpfnWNetCancelJob
 0002:000C       _lpfnWNetCloseJob
 0002:01C0       _lpfnWNetConnectDialog
 0002:01C8       _lpfnWNetConnectionDialog
 0002:003C       _lpfnWNetDeviceMode
 0002:01E4       _lpfnWNetDirectoryNotify
 0002:01C4       _lpfnWNetDisconnectDialog
 0002:0044       _lpfnWNetGetCaps16
 0002:01B0       _lpfnWNetGetConnection
 0002:01E0       _lpfnWNetGetDirectoryType
 0002:0048       _lpfnWNetGetError16
 0002:004C       _lpfnWNetGetErrorText16
 0002:01D0       _lpfnWNetGetPropertyText
 0002:01B8       _lpfnWNetGetUser
 0002:0018       _lpfnWNetHoldJob
 0002:0030       _lpfnWNetLockQueueData
 0002:0008       _lpfnWNetOpenJob
 0002:01CC       _lpfnWNetPropertyDialog
 0002:0038       _lpfnWNetQPoll
 0002:001C       _lpfnWNetReleaseJob
 0002:01B4       _lpfnWNetRestoreConnection
 0002:01DC       _lpfnWNetServerBrowseDialog
 0002:0024       _lpfnWNetSetJobCopies
 0002:01D4       _lpfnWNetShareAsDialog
 0002:01D8       _lpfnWNetStopShareDialog
 0002:0034       _lpfnWNetUnlockQueueData
 0002:002C       _lpfnWNetUnwatchQueue
 0002:0040       _lpfnWNetViewQueueDialog
 0002:0028       _lpfnWNetWatchQueue
 0002:0010       _lpfnWNetWriteJob
 0001:1932       _MapWin32ErrorToWN16
 0001:190A       _MapWNType16To32
 0001:0744       _SetLastError
 0002:0000       _vLastCall
 0002:0002       _vLastError
 0002:03C0       _wAdminCaps
 0002:03C6       _wConnectionCaps
 0002:03CA       _wDialogCaps
 0002:0006       _wDriverVersion
 0002:03C4       _wErrorCaps
 0002:03C8       _wNetTypeCaps
 0002:0004       _wSpecVersion
 0002:03C2       _wUserCaps
 0000:0001  Abs  __acrtused
 0000:0000  Imp  __WINFLAGS           (KERNEL.178)

  Address         Publics by Value

 0000:0000  Imp  __WINFLAGS           (KERNEL.178)
 0000:0000  Imp  GLOBALLOCK           (KERNEL.18)
 0000:0000  Imp  GETPROFILESTRING     (KERNEL.58)
 0000:0000  Imp  WRITEPROFILESTRING   (KERNEL.59)
 0000:0000  Imp  GETMODULEUSAGE       (KERNEL.48)
 0000:0000  Imp  CALLPROC32W          (KERNEL.517)
 0000:0000  Imp  GETPROCADDRESS       (KERNEL.50)
 0000:0000  Imp  GLOBALUNLOCK         (KERNEL.19)
 0000:0000  Imp  GLOBALFREE           (KERNEL.17)
 0000:0000  Imp  LocalInit            (KERNEL.4)
 0000:0000  Imp  INITTASK             (KERNEL.91)
 0000:0000  Imp  LOADLIBRARYEX32W     (KERNEL.513)
 0000:0000  Imp  GETPROCADDRESS32W    (KERNEL.515)
 0000:0000  Imp  LSTRLEN              (KERNEL.90)
 0000:0000  Imp  _LCLOSE              (KERNEL.81)
 0000:0000  Imp  LSTRCMP              (USER.430)
 0000:0000  Imp  LOADLIBRARY          (KERNEL.95)
 0000:0000  Imp  OPENFILE             (KERNEL.74)
 0000:0000  Imp  GETWINFLAGS          (KERNEL.132)
 0000:0000  Imp  LSTRCPY              (KERNEL.88)
 0000:0000  Imp  GLOBALALLOC          (KERNEL.15)
 0000:0001  Abs  __acrtused
 0001:0000       WNETOPENJOB
 0001:0068       WNETCLOSEJOB
 0001:00CA       WNETWRITEJOB
 0001:012C       WNETABORTJOB
 0001:0188       WNETHOLDJOB
 0001:01E4       WNETRELEASEJOB
 0001:0240       WNETCANCELJOB
 0001:029C       WNETSETJOBCOPIES
 0001:02FA       WNETWATCHQUEUE
 0001:035E       WNETUNWATCHQUEUE
 0001:03B6       WNETLOCKQUEUEDATA
 0001:041A       WNETUNLOCKQUEUEDATA
 0001:0472       WNETQPOLL
 0001:04CE       WNETDEVICEMODE
 0001:0524       WNETVIEWQUEUEDIALOG
 0001:0580       WNETGETCAPS16
 0001:05D6       WNETGETERROR16
 0001:062E       WNETGETERRORTEXT16
 0001:0690       WNETGETCAPS
 0001:0704       _GetLanmanDrvEntryPoints
 0001:0744       _SetLastError
 0001:0750       LIBMAIN
 0001:0802       _I_SetCapBits
 0001:0828       WNETADDCONNECTION
 0001:09BE       WNETCANCELCONNECTION
 0001:0A92       WNETGETCONNECTION
 0001:0C2C       WNETRESTORECONNECTION
 0001:0D20       WNETGETUSER
 0001:0E48       WNETBROWSEDIALOG
 0001:0F40       WNETCONNECTDIALOG
 0001:0FE8       WNETDISCONNECTDIALOG
 0001:107E       WNETCONNECTIONDIALOG
 0001:10A0       PRINTCONNECTDIALOG
 0001:1172       WNETPROPERTYDIALOG
 0001:1254       WNETGETPROPERTYTEXT
 0001:1386       WNETSHAREASDIALOG
 0001:1462       WNETSTOPSHAREDIALOG
 0001:153E       WNETSERVERBROWSEDIALOG
 0001:160E       WNETGETDIRECTORYTYPE
 0001:1722       WNETDIRECTORYNOTIFY
 0001:173C       GETLASTERROR32
 0001:17B0       _Get32BitEntryPoints
 0001:190A       _MapWNType16To32
 0001:1932       _MapWin32ErrorToWN16
 0001:19DA       _GetAlignedMemory
 0001:1A3E       _FreeAlignedMemory
 0001:1A5A       WNETPRINTMGRSELNOTIFY
 0001:1A7E       WNETPRINTMGRPRINTERENUM
 0001:1AA2       WNETPRINTMGRCHANGEMENUS
 0001:1AC6       WNETPRINTMGRCOMMAND
 0001:1AEA       WNETPRINTMGREXITING
 0001:1B0C       WNETPRINTMGREXTHELP
 0001:1B32       WNETPRINTMGRMOVEJOB
 0001:1B58       WNETPRINTMGRSTATUSCHANGE
 0001:1B7C       WNETEXITCONFIRM
 0001:1BA0       I_AUTOLOGON
 0001:1BC6       I_LOGOFF
 0001:1BEC       I_CHANGEPASSWORD
 0001:1C10       I_CHANGECACHEPASSWORD
 0001:1C34       I_CONNECTDIALOG
 0001:1C58       I_CONNECTIONDIALOG
 0001:1C7C       WNETCACHEPASSWORD
 0001:1CA0       WNETGETCACHEDPASSWORD
 0001:1CC4       WNETREMOVECACHEDPASSWORD
 0001:1CE8       WNETENUMCACHEDPASSWORDS
 0001:1D0C       WNETSHARESDIALOG
 0001:1D30       WNETSETDEFAULTDRIVE
 0001:1D54       WNETGETSHARECOUNT
 0001:1D78       WNETGETSHARENAME
 0001:1D9C       WNETGETSHAREPATH
 0001:1DC0       WNETGETLASTCONNECTION
 0001:1DE4       WNETGETERROR
 0001:1E30       WNETGETERRORTEXT
 0001:1E78       WNETERRORTEXT
 0001:1EB2       ENABLE
 0001:1EC4       DISABLE
 0001:1ED6       WEP
 0001:1EEA       LFNFINDFIRST
 0001:1F0E       LFNFINDNEXT
 0001:1F32       LFNFINDCLOSE
 0001:1F56       LFNGETATTRIBUTES
 0001:1F7A       LFNSETATTRIBUTES
 0001:1F9E       LFNCOPY
 0001:1FC2       LFNMOVE
 0001:1FE6       LFNDELETE
 0001:200A       LFNMKDIR
 0001:202E       LFNRMDIR
 0001:2052       LFNGETVOLUMELABEL
 0001:2076       LFNSETVOLUMELABEL
 0001:209A       LFNPARSE
 0001:20BE       LFNVOLUMETYPE
 0001:20E2       PmIpx2fHandler
 0001:2111       PmIpx73Handler
 0001:214D       PmIpxEntryPoint
 0001:21A1       LibEntry
 0001:21D3       GRABINTERRUPTS
 0002:0000       _vLastCall
 0002:0002       _vLastError
 0002:0004       _wSpecVersion
 0002:0006       _wDriverVersion
 0002:0008       _lpfnWNetOpenJob
 0002:000C       _lpfnWNetCloseJob
 0002:0010       _lpfnWNetWriteJob
 0002:0014       _lpfnWNetAbortJob
 0002:0018       _lpfnWNetHoldJob
 0002:001C       _lpfnWNetReleaseJob
 0002:0020       _lpfnWNetCancelJob
 0002:0024       _lpfnWNetSetJobCopies
 0002:0028       _lpfnWNetWatchQueue
 0002:002C       _lpfnWNetUnwatchQueue
 0002:0030       _lpfnWNetLockQueueData
 0002:0034       _lpfnWNetUnlockQueueData
 0002:0038       _lpfnWNetQPoll
 0002:003C       _lpfnWNetDeviceMode
 0002:0040       _lpfnWNetViewQueueDialog
 0002:0044       _lpfnWNetGetCaps16
 0002:0048       _lpfnWNetGetError16
 0002:004C       _lpfnWNetGetErrorText16
 0002:01A8       _lpfnWNetAddConnection
 0002:01AC       _lpfnWNetCancelConnection
 0002:01B0       _lpfnWNetGetConnection
 0002:01B4       _lpfnWNetRestoreConnection
 0002:01B8       _lpfnWNetGetUser
 0002:01BC       _lpfnWNetBrowseDialog
 0002:01C0       _lpfnWNetConnectDialog
 0002:01C4       _lpfnWNetDisconnectDialog
 0002:01C8       _lpfnWNetConnectionDialog
 0002:01CC       _lpfnWNetPropertyDialog
 0002:01D0       _lpfnWNetGetPropertyText
 0002:01D4       _lpfnWNetShareAsDialog
 0002:01D8       _lpfnWNetStopShareDialog
 0002:01DC       _lpfnWNetServerBrowseDialog
 0002:01E0       _lpfnWNetGetDirectoryType
 0002:01E4       _lpfnWNetDirectoryNotify
 0002:01E8       _lpfnGetLastError32
 0002:01EC       _lpfnClosePrinter
 0002:01F0       _lpfnConnectToPrinter
 0002:03C0       _wAdminCaps
 0002:03C2       _wUserCaps
 0002:03C4       _wErrorCaps
 0002:03C6       _wConnectionCaps
 0002:03C8       _wNetTypeCaps
 0002:03CA       _wDialogCaps

Program entry point at 0001:21a1
